:020000040000FA
:020000000428D2
:08000800FF30A100FF30A2004F
:10001000E02019149914191599130030F020A11536
:10002000EF200030EA20A401A501A601A7012310BA
:10003000E920A310E8202312E620A312E5202311D3
:10004000E7200A30A7202820282044202528272818
:10005000C830A8002316E6200130C7202312E6206E
:100060000F30AE20A80B2A280430A720C830A800E3
:100070002316E6200130C7202312E6201430AE20DC
:10008000A80B38280430A728851D4728502823119D
:100090002408250203184D282315E720A50A442823
:1000A000A60A2608013C031D57282314E920260828
:1000B000023C031D5D28A314E8202608043C031D10
:1000C0007B2823302702A9000630AA00F520A800CB
:1000D0002808FF3CA4001930270203187028A40147
:1000E0002830270203187628FF30A4002708413C57
:1000F00003187B28A401A70185197F288E28A70A49
:100100002708C83C031D8528A601231124082502C1
:1001100003188B282315E720A50A7C282310E92043
:10012000A310E8202608013C031DA6282312E62080
:10013000A312E520303027020318A0282316E6205A
:1001400027083A3C0318A628A316E5200800A800B3
:100150002808AA006430AB000A30B528A900290895
:10016000AA000130AB000130B528AC00FF30AD0073
:100170002B08AF002A08AE0017302D070318BD2842
:10018000AE0BBC28AF0BBA28AC0BB8280800A900EE
:100190002908AA00AA08031DCE28D2280A30D32095
:1001A000AA03CA280800AB00F430AC00FC30AD0054
:1001B0002B082C07031C00342D070318DC2808002B
:1001C0008316FF23900083120800EC28EC28EC280B
:1001D000EC28EC28A300EC28230885000800F2286E
:1001E000A100F228210865000800AA00AB012A0836
:1001F000003C031CFC2802292908AB0701302A0215
:08020000AA00F7282B080800F2
:02400E0084111B
:00000001FF
